:020000040800F2
:100000000004022001020008F50D0008F50D0008AB
:10001000F50D0008F50D0008F50D0008F50D0008B8
:10002000F50D0008F50D0008F50D0008BD2F0008BE
:10003000F50D0008F50D0008F50D0008F50D000898
:10004000F50D0008F50D0008F50D0008F50D000888
:10005000F50D0008F50D0008F50D0008F50D000878
:10006000F50D0008F50D0008F50D0008F50D000868
:10007000F50D0008F50D0008F50D0008F50D000858
:10008000F50D0008F50D0008F50D0008F50D000848
:10009000F50D0008F50D0008F50D0008F50D000838
:1000A000F50D0008F50D0008F50D0008F50D000828
:1000B00035260008F50D0008F50D0008F50D0008BF
:1000C000F50D0008F50D0008F50D0008F50D000808
:1000D000F50D0008F50D0008B9270008F50D00081A
:1000E000F50D0008F50D0008F50D0008F50D0008E8
:1000F000F50D0008F50D0008F50D0008F50D0008D8
:10010000F50D0008F50D0008F50D0008F50D0008C7
:10011000F50D0008F50D0008F50D0008F50D0008B7
:10012000F50D0008F50D0008F50D0008F50D0008A7
:10013000F50D0008F50D0008F50D0008F50D000897
:10014000F50D0008F50D0008F50D0008AD230008B9
:10015000F50D0008F50D0008F50D0008F50D000877
:10016000F50D0008F50D0008F50D0008F50D000867
:10017000F50D0008F50D0008F50D0008F50D000857
:10018000F50D0008F50D0008CD270008F50D000855
:10019000F50D0008F50D0008F50D0008F50D000837
:1001A000F50D0008F50D0008F50D0008F50D000827
:1001B000F50D0008F50D0008F50D0008F50D000817
:1001C000F50D0008F50D0008F50D0008F50D000807
:1001D000F50D0008F50D0008F50D0008F50D0008F7
:1001E000F50D0008F50D0008F50D0008F50D0008E7
:1001F000F50D0008F50D0008F50D0008F50D0008D7
:1002000072B6374880F3098836484EF60851CEF268
:100210000001086040F20000CCF200004EF634719C
:10022000CEF200010860BFF34F8FBFF36F8F40F233
:100230000000C0F2F0004EF68851CEF200010860D6
:10024000BFF34F8FBFF36F8F4FF00000E1EE100A46
:100250004EF63C71CEF200010860062080F314884F
:10026000BFF36F8F00F06CFD02F064FB4FF0553070
:100270001D491E4A91423CBF41F8040BFAE71C4954
:10028000174A91423CBF41F8040BFAE719491A4A50
:100290001A4B9A423EBF51F8040B42F8040BF8E7A0
:1002A00000201749174A91423CBF41F8040BFAE776
:1002B00000F086FD02F040FB134C144DAC4203DA13
:1002C00054F8041B8847F9E700F03EF8104C114D34
:1002D000AC4203DA54F8041B8847F9E700F06EBD1E
:1002E0000008022000000008000002200004022094
:1002F00000040220783D0008000802205008022077
:1003000050080220502B02200002000800020008C2
:1003100000020008000200082DE9F04F2DED108AC0
:10032000C1F80CD0D0F80CD0BDEC108ABDE8F08F2D
:10033000002383F311882846A047002000F05EFFC9
:1003400000F0F8FE00DFFEE770B51D4C78230025B5
:1003500023706FF07F061E236570A570E570257110
:100360006571A571E57125726672A372E57200F080
:100370002BFC20B10E2325726672A372E57202F087
:1003800039FD104B984217D00133984241F288341E
:1003900012BF002500240125002002F031FD0DB11F
:1003A00000F054F800F06AFC00F058FB204600F022
:1003B000BBF800F04BF8F9E700242546ECE700BF56
:1003C00050080220010007B008B500F0C5FAA0F1FE
:1003D00020035842584108BD07B5054B02211B8830
:1003E000ADF8043001A800F023FB03B05DF804FB76
:1003F000D439000810B51148C3680BB100F0C6FD30
:100400000F4C104A0D4800234FF47A7100F082FD22
:10041000236813B12368013B2360636813B16368E9
:10042000013B6360084B1B7833B9636823B9022032
:1004300000F0E6FB3223636010BD00BF5C080220C1
:10044000740D0220F5030008700802202DE9F04128
:100450002F4C2368013359D02E4D2F4B2A689A42D6
:1004600054D92E4B9B6803F1006303F5C0339A42C5
:100470004CD2002000F00EFB294B0220187000F037
:10048000BDFB72B6274B1C6026682D68BFF34F8FEB
:10049000BFF36F8F083B0022C3F88420BFF34F8F58
:1004A000D3F880205969C2F3C90421F48031C2F322
:1004B0004E3259615201A70743F6E07E02EA0E0868
:1004C00038462146013948EA000CB1F1FF3FC3F834
:1004D00074C200F14040F5D1203A12F1200FEDD165
:1004E000BFF34F8FBFF36F8FBFF34F8FBFF36F8F8C
:1004F0005A6922F400325A610022C3F85022BFF335
:100500004F8FBFF36F8F86F308882847BDE8F081CF
:100510000080010804800108FF7F010850080220C4
:100520007008022008ED00E02DE9F04FBC4B0546B5
:10053000BC489C680022C2608FB0202282F31188E0
:10054000C26898460AB100F021FD0023B64AB548BA
:100550004FF47A7100F0DEFC002383F31188DFF89A
:10056000E4920DB1C9F80050B04EC9F804303370B0
:100570004FF0FF37012000F041FB002D00F0AF816C
:10058000D9F80030002B40F0AA810FB0BDE8F08F01
:100590000220FFF719FF00283AD1A54B1B88ADF8C0
:1005A0002430022109A800F043FAE3E74FF47A70FF
:1005B00000F0D2F9B0F1000BEFDB0220FFF704FFEF
:1005C0000028EAD00BF1FF300428E6D8DFE800F07D
:1005D00003090E1114000EA8052340F8143D042150
:1005E00001E08F48042100F023FA11E00421914832
:1005F000F9E704219048F6E71C25284600F04CFA5C
:1006000004350990042109A800F012FA2C2DF4D128
:1006100000F02AFBFFF7E0FE5FE10220FFF7D4FEC7
:100620000028BAD0012000F035FA0220307000F026
:10063000E5FA4FF0000B5FFA8BFA504600F042FAF1
:100640000BF1010B044618B1504600F04BFAF2E7EB
:1006500001230220337000F0CFFAD8F808309C4212
:1006600007D2204600F018FA013040F01981043416
:10067000F3E700243470C9F80440C9E70220307061
:1006800000F0BCFA322000F067F9B0F1000B84DB17
:100690001BF0030381D1D8F808100BEB04028A4247
:1006A0003FF67BAFBBF5807F3FF677AF634A9A4654
:1006B000DA4501920FDA4FF47A7000F04DF90390A9
:1006C00003990029FFF669AF019A03990AF802100D
:1006D0000AF1010AECE7C820FFF776FE00283FF494
:1006E0005CAF24B9554B4FF0FF321F681A60534B73
:1006F0002BF0030BA344A3EB040A5C4588D05AF803
:100700000410204600F0CEF9204600F0C5F95AF852
:100710000420904240F0C4800434EEE70220FFF74A
:1007200053FE00283FF439AF4FF0000B5D46D8F878
:1007300008309B4534D2BBF1000F14D17A1C12D083
:1007400009973F494B689BB1002209A8135C6B4095
:10075000DBB2013251F82330042A83EA1525F5D1A2
:100760000BF1040BE3E7584600F096F90990E8E72F
:100770001A46082012F0010F4FEA52021FBF82F002
:100780006D4282F4380282F4034282F02002013882
:10079000F0D141F823200133B3F5807FE8D1D3E7CE
:1007A0000EA840F8285D1AE70EA8002340F8143D73
:1007B000642100F009F900287FF4EFAE0220FFF772
:1007C00003FE00283FF4E9AE099800F09DF90EAB56
:1007D00043F8240D0421184605E70EA8002340F82D
:1007E000143D642100F0F0F800287FF4D6AE02201A
:1007F000FFF7EAFD00283FF4D0AE099800F092F927
:100800000EAB43F8200DE5E70220FFF7DDFD0028E1
:100810003FF4C3AE00F08CF90EAB43F81C0DD9E7E2
:10082000500802205C080220F5030008700802202E
:10083000D639000854080220580802207408022003
:1008400074090220740D02200220FFF7BDFD00286C
:100850003FF4A3AE09A9142000F070F905460EA8D4
:10086000042140F8185D00F0E3F8294609A8BAE62B
:100870004FF47A70FFF7A8FD00283FF48EAE7B1C82
:1008800005D1FFF7A9FD324800F0BEFC7DE63946F0
:10089000002000F007F9002000F0FEF88742F0D0B9
:1008A0002C4B7BE60EA8002340F8143D642100F099
:1008B0008BF800287FF471AE0220FFF785FD002839
:1008C0003FF46BAEFFF788FD41F2883000F09CFCEE
:1008D000099800F015FA00F0C7F900254AE6002053
:1008E00000F03AF80390039B002BFFF646AE012080
:1008F00000F082F9039B213B122B3FF63BAE01A295
:1009000052F823F091050008AD0500081B06000809
:100910007505000875050008750500087D060008C6
:10092000750500081D070008A9070008DB07000877
:100930000908000875050008490800087505000841
:10094000710800081106000875050008A5080008D0
:10095000A0860100D83900082DE9F34702AE002433
:100960004FF47A7506F8014D144FDFF8588045436F
:1009700097F900305A1C5FFA84F901D0A34212D1D2
:1009800058F8240003680122D3F81CA031462B46F6
:10099000D047012807D10A4B9DF8070083F8009043
:1009A00002B0BDE8F0870134032CE1D14FF4FA70B6
:1009B00000F02AFC4FF0FF30F2E700BF00080220F1
:1009C000980D0220E43900082DE9F0474FF47A75BC
:1009D000144FDFF8588006464D43002497F9003045
:1009E0005A1C5FFA84F901D0A34210D158F82400B0
:1009F00003680422D3F81CA031462B46D0470428B4
:100A000005D1094B83F800900020BDE8F087013440
:100A1000032CE3D14FF4FA7000F0F6FB4FF0FF30F7
:100A2000BDE8F08700080220980D0220E439000894
:100A300030B4074B1A78074B53F8224023689D695E
:100A4000054B0A46AC460146204630BC604700BF15
:100A5000980D0220E4390008A0860100F8B502F0E4
:100A6000EDF8094C094E0A4F2070002530682378B4
:100A7000834207D902F0DCF8336805440133BD42F4
:100A80003360F3D9F8BD00BF990D02207C0D022020
:100A9000FF7F010002F09AB900F1006000F5C0305C
:100AA0000068704707B502AB00F1006043F8041D11
:100AB0000422194600F5C03002F016F903B05DF8C3
:100AC00004FB0000054B1A68054B1B781344834256
:100AD00002D9104402F0ACB8002070477C0D02200F
:100AE000990D022038B5074D04462868204402F0CD
:100AF000A7F828B928682044BDE8384002F0B8B803
:100B000038BD00BF7C0D022010F0030308D1B0F502
:100B1000806F05D800F10050A0F571200068704783
:100B200000207047014BC058704700BF20F4F01FF1
:100B3000014B1868704700BF002004E0F0B5204B5F
:100B40001E68204B1F885D6893F90840C6F30B02AE
:100B5000BA424FEA164622D09F89BA4221D01F8B53
:100B6000BA4206D102220C2404FB02335D6893F9D9
:100B70000840B6F5805F16D041F201039E4208BFDF
:100B80005A24421E0A44013D0B46934215D215F9E0
:100B9000016F581C4EB1034600F8016CF5E70022C6
:100BA000E1E70122DFE74124EBE72C2582421D70BB
:100BB00001D9981C5C70401AF0BD1846FBE700BFD5
:100BC000002004E004080220094B5B88B3F5805F35
:100BD00009D041F20102934207D10122054B03EBF8
:100BE0008203D87870470022F8E70020704700BFE2
:100BF000002004E0DC390008704700007047000066
:100C00007047000010B50023934203D0CC5CC4545D
:100C10000133F9E710BD000030B5441E14F9010F8F
:100C20000B4660B193F90050854201F1010106D1F4
:100C30001AB993F90020801A30BD013AEEE7002A74
:100C4000F7D1104630BD000002460346981A13F94A
:100C5000011B0029FAD1704702440346934202D097
:100C600003F8011BFAE77047024B1A78024B1A701F
:100C7000704700BF980D02200008022038B5194CBB
:100C8000194D204600F0DCFB2946204600F004FC0C
:100C90002B681648DA6ED2F8043843F00203C2F823
:100CA000043800F0B1FA1249286800F00FFD2B68F3
:100CB0001048DA6E1049D2F8043823F00203C2F863
:100CC0000438A0424FF4E1330B6001D000F01EFB6A
:100CD0000A48A04204D00849BDE8384000F016BBDD
:100CE00038BD00BFF8210220383C000840420F0008
:100CF000A03C000830110220800D02209411022037
:100D000038B50B4B1A780B4B53F822400A4B9C42D8
:100D100005460CD0094B002118461822FFF79CFF0E
:100D2000056001462046BDE8384000F0EFBA38BD06
:100D3000980D0220E4390008F8210220800D0220DD
:100D4000F0B5BFF34F8FBFF36F8F1B4B0021C3F87C
:100D500050125A6942F400325A61BFF34F8FBFF309
:100D60006F8FC3F88410BFF34F8FD3F88020C2F386
:100D7000C904C2F34E325201A50743F6E07602EAF7
:100D8000060E284621464EEA00070139C3F8607274
:100D90004F1C00F14040F6D1203A12F1200FEED165
:100DA000BFF34F8F5A6942F480325A61BFF34F8FBD
:100DB000BFF36F8FF0BD00BF00ED00E0FEE7000065
:100DC000084A094B09498B4204D3094A002193423E
:100DD00005D3704752F8040F43F8040BF3E743F8C8
:100DE000041BF4E7C43D0008502B0220502B0220C6
:100DF000502B02201EF0040F0CBFEFF30880EFF31E
:100E000009808169004A1047110E000870470000F0
:100E1000204B02681A60204B42681A601F4B8268A0
:100E20001A601F4BC2681A601E4B02691A601E4B83
:100E300042691A601D4B82691A601D4BC2691A60B3
:100E40001C4B1D491A681D4B1A601A68120A0A7059
:100E50001A681B4B1A701B4B1A681B4B1A601B4BF2
:100E60001A681B4B1A601B4B1A681B4B1A601B4BF2
:100E70001A681B4B1A601B4B1A681B4B1A601B4BE2
:100E80005A6A1B4B1A601B4B1B68DB0701D500BE5F
:100E9000FEE7FEE7CC0D0220D00D0220D80D022087
:100EA000DC0D0220D40D0220C00D0220C40D022052
:100EB000C80D022028ED00E0A40D0220A80D02209C
:100EC000B80D02202CED00E0B00D022030ED00E066
:100ED000AC0D02203CED00E09C0D022034ED00E062
:100EE000B40D022038ED00E0A00D022000ED00E07E
:100EF000BC0D0220F0ED00E0054B03F114025A6135
:100F00009A614FF0FF32DA6100221A62704700BF27
:100F1000E00D0220F8B503614FF08043C2605C6AC7
:100F2000194B1A46022952F8145F38BF0221954224
:100F300006461F460AD1586198611C6205604560EB
:100F400081600819BDE8F84000F09CBB186AAB68E6
:100F5000241A0C1902D3E41A2D6804E09C4202D230
:100F6000204400F09DFBAB689C42F4D86B68736032
:100F700035601E606E60B460A9684FF0FF33091BD6
:100F8000A960FB61F8BD00BFE00D022010B41B4C4E
:100F9000234653F8141F814210D0416802680A604A
:100FA000026851609A424FF00001C16003D093681B
:100FB00081680B4493605DF8044B70470A68626176
:100FC00000209A425360C86003D15DF8044B00F0E2
:100FD00061BB93688868034493604FF08042506A15
:100FE000226A821A9342E6D99B1A022B2CBFC018A0
:100FF00002305DF8044B00F053BB00BFE00D02204F
:10100000024B00221B605B609A607047E00D02207B
:10101000002303748268054B1B6899689142FBD2D8
:101020005A6803604260106058607047E00D02200B
:1010300008B5202383F31188037C032B05D0042BF0
:101040000DD02BB983F3118808BD436900221A60C3
:101050004FF0FF334361FFF7DBFF0023F2E790E837
:101060000C001A6002685360F2E70000002303746A
:101070008268054B1B6899689142FBD85A680360E7
:101080004260106058607047E00D0220054B1969FE
:101090000874186802681A605360186101230374A9
:1010A000FFF73AB9E00D022030B54B1C87B005467A
:1010B0000A4C10D023690A4A01A8FFF72BFF2846E3
:1010C000FFF7E4FF049B13B101A8FFF75FFF23695B
:1010D000586907B030BDFFF7D9FFF8E7E00D0220EF
:1010E0003110000838B50C4D41612B6981689A6850
:1010F0009142044603D8BDE83840FFF789BF18463F
:10110000FFF786FF01232C61014623742046BDE8CA
:101110003840FFF701B900BFE00D0220044B1A6808
:101120001B6990689B68984294BF0020012070471B
:10113000E00D022010B5084C236820691A6822606F
:101140005460012223611A74FFF790FF0146206961
:10115000BDE81040FFF7E0B8E00D022008B5FFF74A
:10116000DDFF18B1BDE80840FFF7E4BF08BD00008F
:101170008260022202740022427482617047000081
:101180008368A3F1840243F8142C026943F8442CC9
:10119000426943F8402C084A43F8242CC26843F8BB
:1011A000182C022203F8102C002203F80F2C43F80D
:1011B000082CA3F1200070473103000808B5FFF7A1
:1011C000DFFFBDE80840FFF723BF000010B5202374
:1011D00083F31188FFF7D4FF00210446FFF782FF55
:1011E000002383F31188204610BD0000024B1B69C9
:1011F00058610F20FFF74ABFE00D0220202383F340
:101200001188FFF7F3BF000008B50146202383F3E0
:1012100011880820FFF748FF002383F3118808BDD9
:1012200010B5054C2369036058610320FFF72EFFBA
:101230002369586910BD00BFE00D022003682BB17F
:101240000022026059611846FFF7E2BE70470000B5
:1012500049B1064B42681B6918605A6013604360CD
:101260000420FFF721BF4FF0FF307047E00D022050
:101270000368984206D01A680260506059611846A7
:10128000FFF7C6BE7047000038B504460D4620681B
:10129000844200D138BD036823605C604561FFF77C
:1012A000B7FEF4E70C3002F021B900004FF0FF3335
:1012B0000C3002F01BB90000303002F0B7B900006A
:1012C0004FF0FF33303002F0B1B900000C3002F0C3
:1012D000E7B800004FF0FF310C3002F0E1B8000039
:1012E000303002F061B900004FF0FF32303002F0D0
:1012F0005BB9000001F074BA0346034A43F8042BBB
:1013000043600123037270471C3A000810B5202384
:10131000044683F3118801F0B9FA022323720023F3
:1013200083F3118810BD000038B5436904460D46AB
:101330001BB90421084401F01DFE294604F10C00EC
:1013400002F092F8002806DA201D4FF48061BDE813
:10135000384001F00FBE38BD13B5446BD4F88C345F
:101360001A681178042916D1217A022913D1197922
:10137000128901238B4013420DD101A904F14400CD
:1013800001F07AFF024630B1D4F88C44019B2179F8
:10139000206800F0EBF902B010BD00000C3001F045
:1013A000E9BE00004FF0FF330C3001F0E3BE000057
:1013B000443001F0CDBF00004FF0FF33443001F066
:1013C000C7BF00000C3001F0B7BE00004FF0FF3186
:1013D0000C3001F0B1BE0000443001F099BF0000B4
:1013E0004FF0FF32443001F093BF0000D0F88C245E
:1013F00038B5136819780429054601D0012038BD95
:10140000017A0229FAD112795C89012090400440C6
:10141000F4D105F10C0001F049FE02460028EDD0A0
:10142000D5F88C544FF480732868697900F08CF9F2
:10143000204638BD406BFFF7D9BF00007047000061
:101440007FB50346114A43F8042B01254360022669
:101450000F4B057204460290019300F17C0229466D
:1014600000964FF480730C3001F0FCFD094B0193A2
:10147000029400964FF4807304F52172294604F11A
:10148000440001F0D5FE04B070BD00BF3C3A000836
:1014900035140008591300080B68202282F31188C4
:1014A0000A7903EB820210624A790D3243F8220076
:1014B0008A7912B103EB8203186202230372C0F827
:1014C0008C14002383F311887047000038B504465C
:1014D00001250221043001F04DFD04F10C002575B9
:1014E0006FF00101FFF7D0FE84F84C5004F1440086
:1014F0006FF00101BDE83840FFF7C6BE10B501210D
:101500000446043001F036FD0023237584F84C3086
:1015100010BD000038B5044600250C3001F0BAFDBE
:1015200004F14400257501F09BFE201D84F84C5009
:10153000012101F01FFD2046BDE83840FFF756BFEE
:1015400090F85C3003F06003202B19D190F85D20F7
:10155000212A0AD0222A4FF000030ED0202A0FD1D0
:10156000084A02650722426504E0064B036507232B
:101570004365002383650120704703654365F9E7F0
:101580000020704728080220D0F88C3437B51A683C
:101590001178042904461AD1017A022917D1197940
:1015A000128901238B40134211D100F144052846D2
:1015B00001F02CFF58B101A9284601F05DFED4F8D6
:1015C0008C44019B21790246206800F0CFF803B0DB
:1015D00030BD000000EB8103F7B51C6A05460E46DE
:1015E000F4B1202383F3118805EB8607201D082121
:1015F00001F0C0FCFB685B691B68443413B12046F2
:1016000001F048FE01A9204601F036FE024648B12D
:10161000019B3146284600F0A9F8002383F3118886
:1016200003B0F0BDFB685A691268002AF5D01B8A26
:10163000013B1340F1D105F15C02EAE70D3110B531
:1016400050F82140CCB1202383F311880421601885
:1016500001F090FCD4F88C241368527903EB8203D8
:1016600004F10C00DB689B69596801F029FD2046F4
:10167000FFF7BCFE002383F3118810BD7047000004
:1016800000F0ECBF4FF08043002258631A61022241
:10169000DA6070474FF080430022DA607047000044
:1016A0004FF080435863704700F0A4BB01230370E0
:1016B0000023436000F1240200F1380142F8043BAA
:1016C0008A421361FAD103814381704738B50446D9
:1016D000202383F3118800254160C56005614561C1
:1016E0008561C561056200F099FB0223237085F3D3
:1016F000118838BD70B500EB810305465069DA608A
:101700000E46144618B110220021FFF7A5FAA06971
:1017100018B110220021FFF79FFA31462846BDE894
:10172000704000F055BC0000028902F00102028105
:10173000428902F00102428100220261426182611B
:10174000C261026200F0D8BCF0B400EB81044789AA
:10175000E4680125A4698D403D4345812360002351
:10176000A2606360F0BC00F0F3BC0000F0B400EBDA
:1017700081040789E468012564698D403D43058142
:1017800023600023A2606360F0BC00F071BD000024
:1017900070B50223002504460370A0F8645080F859
:1017A000665080F8675005814581C56005614561D7
:1017B0008561C561056280F84C5000F0A7FB636845
:1017C0001B6823B129462046BDE87040184770BD0C
:1017D000436802781B6880F86820052202700BB10C
:1017E0000421184770470000436890F868201B6880
:1017F00002700BB1052118477047000070B5002337
:10180000044680F84C3000F15C0200F097FC6368FD
:101810009B685BBB94F85C5015F0600614D194F89B
:101820005D3005F07F0545EA0325B5F5407F00F002
:10183000A58059D8022D00F0F1803FD8002D00F08E
:101840008780012D00F0E4800021204600F0D4FEC6
:101850000021204600F0C6FE63681B6813B1062114
:1018600020469847062384F84C3070BD20469847A0
:101870000028CFD094F8632094F8623043EA022322
:10188000626D934238BF636594F95C30656D002BDF
:101890004FF0200380F20181002D00F0F080012242
:1018A00084F84C2083F311880021636D226D20465B
:1018B000FFF75CFF002383F3118870BDB5F5807FCF
:1018C0004DD0B5F5817FBFD194F85E30002BBBD1F0
:1018D00094F8603013F00F0126D01A06204640F12C
:1018E000B78000F09DFE1FE0B5F5C06F50D020D846
:1018F00040F202339D4200F0AE80B5F5A06FA3D157
:10190000B4F85C30B3F5A06F0ED194F85E3084F873
:101910006630204600F050FB63681B6813B101215C
:101920002046984703232370002323656365A3653E
:10193000A0E7B5F5106F41D040F602439D4267D055
:10194000B5F5006F80D104F167032365012333E00F
:1019500004F16403236502236365A5658AE794F8AF
:101960005E30012B7FF470AFB4F8643023F00203D3
:10197000A4F8643026656665A6657BE794F85E305A
:10198000012B7FF461AFB4F8643043F00203EFE75A
:1019900094F86120616894F860304D6894F85F10A5
:1019A00043EA0223204694F85E20A84700283FF42B
:1019B0004BAF4368236503686365DDE794F86720F0
:1019C00094F85E309A42AFD02378042B10D12023B4
:1019D00083F311882046FFF7A7FE86F3118863681A
:1019E00084F867601B68032121700BB1204698477B
:1019F00094F85E30002B97D084F86730042323706E
:101A000063681B68002B8FD00221204698478BE724
:101A10002E4B236502236365002388E794F860104A
:101A200011F0800F204601F00F010ED000F078FB7E
:101A3000012806D002287FF407AF254B2365606597
:101A40009AE7244B2365656596E700F05BFBEFE7BB
:101A500000F0DCFD68E794F85E30002B7FF4F4AE14
:101A600094F8603013F00F013FF45EAF1B06204680
:101A700002D500F0C1FD57E700F0B4FD54E70322A2
:101A800084F84C2083F311882B462A4629462046A9
:101A9000FFF75AFE85F3118870BD5DB1042284F80A
:101AA0004C2083F311880021636D226D2046FFF7DF
:101AB0004BFEFFE6052284F84C2083F311882B4669
:101AC0002A4629462046FFF751FEE3E7643A00081C
:101AD0005C3A0008603A000838B590F84C3004468B
:101AE000062B22D8DFE803F03704223737323700DD
:101AF00090F8631090F86220436D42EA01229A4206
:101B000014D9C268128AB3FBF2F502FB15356DB920
:101B1000202383F311882B462A462946FFF726FE09
:101B200085F31188022384F84C3038BD032384F8F0
:101B30004C30202383F3118800231A46194620468F
:101B4000FFF702FE002383F3118838BD836D03B1D4
:101B500098470023E7E7002100F04EFD00212046D2
:101B600000F040FD63681B6813B1062120469847CA
:101B70000623D8E790F84C20062A38B5044621D829
:101B80000123934013F0670F1DD113F008050FD107
:101B9000DB0617D5052380F84C30202383F311880A
:101BA0002B462A462946FFF7E1FD85F3118838BD0B
:101BB000C3689B695B682BB9836D03B198470023A9
:101BC00084F84C3038BD002100F016FD002120467D
:101BD00000F008FD63681B6813B106212046984792
:101BE0000623EDE7036F30B500229D68C46E1146F1
:101BF0004FF0FF3004EB421301329542C3F8001955
:101C0000C3F81019C3F80809C3F8001BC3F8101B68
:101C1000C3F8080BEED24FF00113C4F81C3830BDE6
:101C2000890141F02001016103699B06FCD4122067
:101C300001F082B92DE9F04F202387B00446C56E2C
:101C400083F3118800F17C0305934FF0000B237898
:101C5000012B04D0A36F4BB96B69DB0606D4AB69CB
:101C6000059843F01003AB61FFF7DAFA8BF31188A4
:101C70004FF0000E4FF02009236F9B685FFA8EF043
:101C800083421BD2202383F31188E0E7E16E0A6AC6
:101C900002F4F013B3F5802F66D0B3F5402F0DD1C9
:101CA000C2F30A1602F00F0204EB820201F5805122
:101CB000D3681F6A00231A469E4248D1696911F011
:101CC0001001E3D1012303FA00F2A36F1A4200F0DE
:101CD0008C8089F31188AB6823F00103AB60A36F9C
:101CE00023EA0203A36781F3118804EB8003D3F88E
:101CF0000C80D8F814100B680093431C1B0302934C
:101D0000430104934868009B98425FD2B8F8106082
:101D1000E76E1B1AB34228BF3346049EBE19D6F89D
:101D20001869B6B2B3EB860F62D8029EBE1903964D
:101D30008E680196A6F1040A9C46039E5AF8047F19
:101D40003760BCF1040F3BD9ACF1040CF5E713F09C
:101D5000030F08BF0A68072B98BF3A7003F101030D
:101D60009CBF120A0137A7E7C2F30A1602F00F025E
:101D700004EB820201F58051D3689B691F68D3F898
:101D800008805B68A7EB030C00231F469E4208D126
:101D9000D36899698A684B68324433448A604B60DF
:101DA0008CE713F0030F08BF0F689C4588BF88F8C5
:101DB000007003F1010384BF3F0A08F10108E5E761
:101DC000019E1E4403448E604B609BE7012189F312
:101DD0001188AB6843F00103AB6021B9D5F8343802
:101DE0001A43C5F834288BF311880EF1010E43E72E
:101DF0000021ECE710B5074C2046FFF757FC4FF0E9
:101E0000A0420023E266044AE3672267C4F88030F8
:101E100010BD00BF280E02208C3A000870B5037870
:101E2000012B86B005465DD1304BC46E984213D16C
:101E30002F4B5A6B42F080025A635A6942F080027B
:101E40005A6100225A610E21432001F041FC294BC6
:101E5000E360294BC4F800380023AB67C4F8003EA8
:101E6000C02323604FF40413A363EE6E202001F01F
:101E700063F8012333613369DB07FCD4122001F0DE
:101E80005BF83369002BFCDA0026A6602846FFF7D2
:101E9000A9FE6B68C4F81068DB68C4F81468C4F85D
:101EA0001C680BBB154BA3614FF0FF336361D5F882
:101EB00080309BB9124B009305F18803019305F51F
:101EC0003C7302930223039368460E4B04930595DB
:101ED000FFF774F9C5F88000FFF740F9A36843F0F5
:101EE0000103A36006B070BD074BDCE7280E02209B
:101EF000003802404014004003002002003C30C083
:101F0000983A0008351C0008083C30C0F8B5C46E8B
:101F1000054600212046FFF783FE296F00234FF07E
:101F200001128F68C4F834384FF00066C4F81C28DA
:101F30004FF0FF3004EB431201339F42C2F80069B7
:101F4000C2F8006BC2F80809C2F8080BF2D20B689D
:101F50006B676362EB6E10221A611E6916F0100641
:101F6000FBD1122000F0E8FFD4F8003823F4FE6320
:101F7000C4F80038A36943F4402343F01003A3617D
:101F80000923C4F81038C4F81438094BEB60094B26
:101F9000C4F8106BC4F8003BC4F81069C4F80039E9
:101FA0006B6F03F1100243F480136A67A362F8BDFC
:101FB000683A000840800010C26E90F86610D2F8AF
:101FC000003823F4FE6343EA0113C2F80038704777
:101FD0002DE9F0410EB200EB86080D46D8F80C1042
:101FE0000F6807F00303022B50D0032B50D03D4A5B
:101FF0003D4F012B18BF1746C46E4FEA451E04EB38
:102000000E030022C3F8102B8A6905F1100C002A78
:1020100040D04A8A05F158035B013A43E25001235C
:10202000D4F81C2803FA0CF31343A6444A69C4F8F5
:102030001C380023CEF8103905F13F03002A39D0AF
:102040000A8A898B9208012988BF4A43416F04EBB1
:102050008303561841EA0242466729465A602046E1
:10206000FFF7DEFDD8F80C301B8A43EA85531F4387
:1020700005F148035B01E7500123D4F81C2803FA5B
:1020800005F51543C4F81C58BDE8F081174FB3E7B8
:10209000174FB1E704EB4613D3F8002B22F40042AC
:1020A000C3F8002BD4F81C28012303FA0CF322EA0E
:1020B0000303BAE704EB83030E4A5A6004EB4616A7
:1020C00029462046FFF7ACFDD6F8003923F400433B
:1020D000C6F80039D4F81C38012202FA05F523EAC3
:1020E0000505CFE700800010008004100080081074
:1020F00000800C1000040002026F12684267FFF7B4
:1021000071BD00005831C36E49015B5813F40040A3
:1021100004D013F4001F14BF0120022070470000F8
:102120004831C36E49015B5813F4004004D013F4E6
:10213000001F14BF012002207047000000EB810146
:10214000CB68196A0B6813604B68536070470000D6
:1021500000EB810330B5DD68AA691368D36019B953
:10216000402B84BF402313606B8A1468C26E1C44EA
:10217000013CB4FBF3F46343033323F0030302EBAA
:10218000411043EAC44343F0C043C0F8103B2B68FE
:1021900003F00303012B09B20ED1D2F8083802EB89
:1021A000411013F4807FD0F8003B14BF43F08053FC
:1021B00043F00053C0F8003B02EB4112D2F8003B61
:1021C00043F00443C2F8003B30BD00002DE9F0416C
:1021D000264DEE6E06EB40130446D3F8087BC3F899
:1021E000087B38070AD5D6F81438190706D505EB49
:1021F00084032146DB6828465B689847FA0733D595
:10220000D6F81438DB072FD514B995F84C305BB3EA
:1022100005EB8403D968CCB98B69488A5E68B6FB44
:10222000F0F200FB12628AB91868DA6890420DD2A7
:10223000121A83E81400202383F311880B482146E7
:10224000FFF786FF84F31188BDE8F081012303FACC
:1022500004F26B8923EA02036B81CB6823B1214628
:102260000248BDE8F0411847BDE8F081280E022081
:1022700000EB810370B5DD68C36E6C692668E660AB
:102280004A0156BB1A444FF40020C2F810092A68CC
:1022900002F00302012A0AB20ED1D3F8080803EBB8
:1022A000421410F4807FD4F8000914BF40F080502D
:1022B00040F00050C4F8000903EB4212D2F80009C4
:1022C00040F00440C2F80009D3F83408012202FAB1
:1022D00001F10143C3F8341870BD19B9402E84BF11
:1022E0004020206020682E8A841940F00050013C74
:1022F0001A44B4FBF6F440EAC440C6E72DE9F041C5
:10230000284CE66E06EB40130546D3F80879C3F86F
:102310000879F9071AD5D6F81038DA0716D504EB7C
:102320008003D9684B691868DA6890422CD2121A77
:102330004FF000081A60C3F80480202383F311884B
:1023400029462046FFF794FF88F311883B0619D5EC
:10235000D6F83428012303FA05F5154212D02023BC
:1023600083F31188A36F10482B43A367D6F8343842
:1023700023EA0505C6F834580021FEF75FFF002365
:1023800083F31188BDE8F081012303FA05F2238964
:1023900023EA020323818B68002BD7D029462046ED
:1023A0009847D3E7280E0220A40E02202DE9F74F0C
:1023B0008A48C46E6669A3691E4016F4805F666130
:1023C000054608D000238367FFF7E2F903B0BDE8B4
:1023D000F04F00F005BE002E12DAD4F8003E7F4820
:1023E00099071EBFD4F8003E23F00303C4F8003E53
:1023F000D4F8043843F00103C4F80438FFF7F4F9C3
:10240000320504D500237548AB67FFF7E1F9B30443
:102410000CD5D4F8083813F0060FE36823F4705392
:102420000CBF43F4105343F4A053E360370704D5C3
:102430006B68DB680BB169489847F00262D4B1025F
:102440000CD5D5F86C80DFF894A100274FF0010976
:102450002B6F9B68F9B28B4280F0A380F2060DD5FA
:10246000202383F31188A3695D4823F01003A3613F
:102470000021FEF7E3FE002383F311883303D4F831
:1024800018481DD5E70302D50020FFF79FFEA503DE
:1024900002D50120FFF79AFE600302D50220FFF764
:1024A00095FE210302D50320FFF790FEE20202D53C
:1024B0000420FFF78BFEA30202D50520FFF786FE5E
:1024C000770383D5E60702D50020FFF717FFA5079E
:1024D00002D50120FFF712FF600702D50220FFF7A7
:1024E0000DFF210702D50320FFF708FFE20602D502
:1024F0000420FFF703FFA3067FF568AF0520FFF771
:10250000FDFE63E7D5F86CA0DFF8D4B04FF000090A
:102510002B6F9B685FFA89F7BB4290D30AEB471396
:10252000D3F8002902F44022B2F5802F36D1D3F837
:102530000029002A32DAD3F8002942F09042C3F889
:102540000029D3F80029002AFBDB3946E86EFFF7A3
:1025500067FB01232A89BB406FEA030808EA0202ED
:102560002A8105EB8702D268926822B139461B485E
:1025700001939047019B202282F31188DAF83428D6
:1025800008EA0202CAF83428AA6F00211343584609
:10259000AB67FEF753FE002383F3118809F10109AD
:1025A000B6E708EB4112D2F8003B03F44023B3F541
:1025B000802F10D1D2F8003B002B0CDA6A8909FA7F
:1025C00001F322EA03036B8105EB8103DB68DB681F
:1025D0000BB15046984701373AE700BF280E02205A
:1025E000A40E0220C36E03EB4111D1F8003B43F46B
:1025F0000013C1F8003B7047C36E03EB4111D1F8E3
:10260000003943F40013C1F800397047C36E03EB7F
:102610004111D1F8003B23F40013C1F8003B70478F
:10262000C36E03EB4111D1F8003923F40013C1F854
:10263000003970474FF0804310B51A69920708D5EA
:1026400000241C61202383F3118800F03BFC84F3F9
:102650001188BDE8104000F0C3BC00000E4A136CA6
:1026600043F0010313640D4A936843F00103936040
:102670004FF080436B229A624FF0FF32DA62002201
:102680009A615A63DA605A6001225A6108211A601D
:102690001C2001F01DB800BF00380240002004E0FB
:1026A000024A136843F080031360704700440040FF
:1026B000024A136843F080031360704700780040BB
:1026C0002DE9F041466D3768F56935620446280703
:1026D00019D015F0080F0CBF00218021EA0748BF70
:1026E00041F02001AB0748BF41F04001680748BFF7
:1026F00041F48071202383F31188201D00F03AFCFF
:10270000002383F31188EA050AD5202383F3118877
:102710004FF40071201D00F02DFC002383F311887D
:10272000AB060CD5202383F31188736A94F85C10F0
:1027300020461940FEF7F8FD002383F31188380680
:1027400016D5290614D5202383F3118804F130000F
:1027500000F052FF002825DA0821201D00F00AFCB5
:1027600027F0C00343F040033360002383F3118854
:102770006A060ED5202383F31188626CA36C9A42FB
:1027800001D1A36B83B927F040073760002383F39F
:102790001188EB060DD5226E136953B15069BDE85F
:1027A000F0411847B062E0E71021201D00F0E2FB85
:1027B000E9E7BDE8F081000008B50348FFF780FFB6
:1027C000BDE8084000F00CBC3011022008B50348F9
:1027D000FFF776FFBDE8084000F002BC941102202C
:1027E00037B51F4C1F4D2046FEF786FD009404F1BF
:1027F0000C0000234FF480621B4900F027FE4FF4C9
:102800008062009404F13000184B194900F0C0FEBA
:10281000184B6365A565184C0B21262000F058FF66
:102820002046FEF769FD04F10C00009400234FF4EC
:102830008062124900F00AFE04F130000094104B4F
:1028400010494FF4806200F0A3FE0F4B63650B212B
:102850005220A56503B0BDE8304000F039BF00BF8D
:102860003011022080F93703F8110220A126000858
:10287000F81902200044004094110220F8150220AB
:10288000B1260008F81D022000780040204B0029E6
:1028900008BF1946037A0166012B10B507D11D4BFD
:1028A000984226D11C4A136C43F400331364426DE2
:1028B0000C68836DB3FBF4F3D3608B6843F0400383
:1028C0005360CB6843F0010393604B6843F4967107
:1028D00041F0010111604FF0FF3111625A0505D539
:1028E00013F010230DD0B3F1805F0ED080F85C1090
:1028F00010BD0A4B9842DAD1074A136C43F080436B
:10290000D4E77F2380F85C3010BD3F23FAE700BF97
:10291000A43A00083011022000380240941102202D
:1029200000207047FEE70000704700004FF0FF30C6
:102930007047000000F00CBF08B500F07FFB00F00E
:102940007BFABDE8084000F0FFB8000070470000C7
:10295000022906D0032906D00129064818BF002005
:10296000704705487047032A9ABF044800EBC2002D
:1029700000207047FC3C0008B03C000830080220F2
:1029800070B5044608460D46FEF75EF9C6B220460D
:10299000013403780BB9184670BD32462946FEF75C
:1029A0003BF90028F3D1012070BD00002DE9F04F64
:1029B00081469BB008460D461646FEF745F93D494F
:1029C000C4B22846FFF7DCFF08B10434E4B23A4948
:1029D0002846FFF7D5FF08B11034E4B2632C01AFED
:1029E0000CD8DFF8E0A0DFF8E0B03C4695F80080B6
:1029F000B8F1000F1CD184F8008003E02946384666
:102A000000F08AFF3846FEF71FF9C0B2431C5B0096
:102A100089E8480033700323737000230236194697
:102A2000DAB2904206F102063DD81BB0BDE8F08F45
:102A3000B8F1250F32D107221E492846FEF7ECF8DF
:102A400070B9DBF800202260DBF804206260BBF87C
:102A5000082022819BF80A20A27207350B34C5E7B3
:102A6000082215492846FEF7D7F8B8B91348A21C22
:102A700010F8011F124B4FEA111E01F00F011EF852
:102A80000AE011F80A1002F802EC984202F8011C60
:102A900002F10202ECD118340835A7E784F800806F
:102AA00001350134A2E7FA5C06F8022C06F8011C95
:102AB0000133B5E7403C0008483C00081FF4F01F14
:102AC0002BF4F01F5D3C0008513C000808B52023A2
:102AD00083F311880348FEF757FD002383F3118821
:102AE00008BD00BFF821022010B50446052916D8FC
:102AF000DFE801F016150316161D202383F3118855
:102B00000E4A0121FEF7F6FD20460D4A0221FEF78E
:102B1000F1FD0C48FEF7FEFC002383F3118810BD85
:102B2000202383F311880748FEF7D0FCF4E7202325
:102B300083F311880348FEF7E1FCEDE7F03B000862
:102B4000143C0008F821022038B50C4D0C4C0D49FE
:102B50002A4604F10800FFF729FF05F1CA0204F133
:102B600010000949FFF722FF05F5CA7204F11800A9
:102B70000649BDE83840FFF719BF00BFB82602205C
:102B800030080220703C0008873C0008483C0008E0
:102B9000BFF34F8F024AD368DB03FCD4704700BFFA
:102BA000003C024008B5074B1B7853B9FFF7F0FF14
:102BB000054B1A69002ABFBF044A5A6002F18832E5
:102BC0005A6008BD16290220003C024023016745D7
:102BD00008B5054B1B7833B9FFF7DAFF034A1369D1
:102BE00043F00043136108BD16290220003C024057
:102BF0000B2870B513D80B4A0B4C137863B90B4EE6
:102C00004FF0006144F8231056F8235001330C2B89
:102C10002944F7D10123137054F8200070BD00201F
:102C200070BD00BF48290220182902201C3D000861
:102C3000014B53F8200070471C3D00080C207047E2
:102C40000B2810B5044601D9002010BDFFF7D0FFB6
:102C5000064B53F824301844C21A0BB9012010BD9A
:102C600012680132F0D1043BF6E700BF1C3D0008BA
:102C70000B2810B504462FD8FFF78AFFFFF792FF05
:102C80001649F323CB60FFF783FFC300DBB243F4A5
:102C9000007343F002030B610B6943F480330B6153
:102CA000FFF776FFFFF7A4FF0D4B53F824300344E2
:102CB000BFF34F8F0B4A98420AD3BFF34F8FBFF336
:102CC0006F8FFFF785FF2046BDE81040FFF7B8BFC4
:102CD000C2F85C022030EEE7002010BD003C02404C
:102CE0001C3D000800ED00E02DE9F047D407154633
:102CF0004DD41318B3F1026F49D2324B1B68DA0777
:102D000045D5314CFFF74EFFF323E360FFF740FF5B
:102D10002F46401A40F20129032F884601EB000696
:102D200018D8294C40F201197B1A4344012B01EBBE
:102D3000000623692FD823F001032361FFF748FF22
:102D40002846BDE8F087366851F8043CB34218D1F4
:102D5000043FE1E7B307E4D1236923F4407323611F
:102D6000236943EA090323610431D8F80030336052
:102D7000BFF34F8FFFF70CFFE368002BE3D0F32383
:102D8000E360236923F001032361FFF721FF4FF084
:102D9000FF30BDE8F08723F440732361236943EAE1
:102DA000090323618A4631F8023B3380BFF34F8F1A
:102DB000FFF7EEFE3688BAF80030B6B2B342B3D0B1
:102DC000DFE700BF00380240003C0240084908B578
:102DD0000B7828B153B9FFF7E5FE01230B7008BD4E
:102DE00023B1BDE808400870FFF7F2BE08BD00BF80
:102DF00016290220014B186D704700BF00280040C3
:102E0000094B1A6F120407D41A6F42F400721A6742
:102E10001A6F42F400421A67044A136843F480733D
:102E20001360034B18657047003802400070004083
:102E300000280040FEE7000010B51A4CFEF7E0F84D
:102E4000FEF75AF800F0AAF8802217492046FEF74C
:102E50008FF9012344F8180C0374144B144AD968F1
:102E600021F4E0610904090C0A431249DA60CA68D6
:102E700042F08072CA60104A1049C2F8B01F11684F
:102E800041F0010111601022DA77202283F822201C
:102E9000002383F3118862B60948BDE81040FEF7AD
:102EA00095B900BF080E02204C3D000800ED00E07F
:102EB0000003FA05F0ED00E0001000E055CEACC5CF
:102EC000543D00082DE9F8431A4C4FF0804300258B
:102ED0006769586A04F114082E46226ABB68811A91
:102EE0008B420CD96169414522D013441B1A022B35
:102EF0002CBFC0180230BDE8F843FEF7D1BB134425
:102F000023623B68D7F80C90C3F8048043456361A3
:102F1000FD6001D1FEF7BEFB86F311883869C84712
:102F2000202383F311884FF080436769586AD4E700
:102F3000BDE8F883E00D0220034B59685A68521A25
:102F40009042FBD8704700BF001000E0836919432E
:102F5000037C81610A2B03D14369194205D1704773
:102F60000B2B06D143698B4303D100234361FEF74A
:102F70004FB8704770B5046805460E46AC4200D1A4
:102F800070BDE3683343E36016B12269134203D096
:102F9000A1686068FFF7DAFF2468EFE7034B044A93
:102FA0001A60044B044A1A60704700BF4C2B022081
:102FB000502B0220482B02200000082080B5074A31
:102FC000536823F0010300AF5360EFF309836833C4
:102FD00083F30988002383F3118880BD30EF00E07C
:102FE00098B5202300AF83F31188104B5B6813F46E
:102FF000006318D0F1EE103AEFF309844FF08073BC
:1030000044F84C3C0A4BDB6844F8083CA4F16803E4
:1030100083F30988FEF782F818B1064B44F8503C58
:1030200098BD054BFAE783F3118898BD00ED00E0E9
:1030300030EF00E0410300084403000808B500F049
:103040005DFB074800F00CFCFEF754F9FEF72CFB83
:10305000FEF7F4F9FFF77AFCBDE80840FEF710BB75
:10306000BC3A000830B5039C0172043304FB03250D
:10307000C361049B03630021059B00604060C16045
:10308000426102618561046242628162C16243639E
:1030900030BD00000022416A41610161C26082626C
:1030A000C2626FF00101FEF7EFB8000003694269E8
:1030B000934203D1C2680AB100207047181D7047BF
:1030C00003691960C2680132C260C269134482692F
:1030D0000361934224BF436A03610021FEF7C8B82D
:1030E00038B504460D46E3683BB16269131D1268AA
:1030F000A3621344E362002038BD237A33B9294622
:103100002046FEF7A5F80028EDDA38BD6FF0010083
:10311000FBE70000C368C269013BC3604369134415
:1031200082694361934224BF436A436100238362FF
:10313000036B03B11847704770B52023044683F32F
:103140001188866A3EB9FFF7CBFF054618B186F3B2
:103150001188284670BDA36AE26A13F8015BA36276
:10316000934202D32046FFF7D5FF002383F3118853
:10317000EFE700002DE9F74F1F4604460E46914643
:10318000202383F311884FF080480025D8F824309D
:10319000FB18009307F1FF3AAB46A36AABB91AF1EB
:1031A000030F06D939462046FFF79AFF68B100237E
:1031B00005E0D8F82410009A511A8F42F3D283F315
:1031C0001188284603B0BDE8F08FA16AE36AA9EB35
:1031D00005025B1A934228BF1346402B1CD9334685
:1031E00001F1400251F8040B43F8040B9142F9D16C
:1031F000A36A40334036A3624035A26AE36A9A422A
:1032000002D32046FFF786FF8BF311884D45D8D2B5
:10321000202383F31188C0E71A4630460193FDF757
:10322000F1FC019BA26A1A441E44A2621D44E4E719
:1032300010B5029C0172043303FB0421C361002317
:103240008362C362039B0363049B00604060C460AD
:1032500042610261816104624262436310BD000009
:10326000026AC260426A4261026100228262C262F4
:103270006FF00101FEF708B8436902699A4203D171
:10328000C2680AB100207047184650F8043B0B6032
:1032900070470000C368C2690133C36043691344C7
:1032A00082694361934224BF436A43610021FDF771
:1032B000DFBF000038B504460D46E3683BB1236923
:1032C0001A1DA262E2691344E362002038BD237A2A
:1032D00033B929462046FDF7BBFF0028EDDA38BD9B
:1032E0006FF00100FBE7000003691960C268013A52
:1032F000C260C269134482690361934224BF436A76
:10330000036100238362036B03B118477047000019
:1033100070B5202304460E4683F31188856A35B9BB
:103320001146FFF7C7FF10B185F3118870BDA36A7E
:103330001E70A36AE26A01339342A36204D3E16977
:1033400020460439FFF7D0FF002080F3118870BDBC
:103350002DE9F74F1F4604460D469146202383F37F
:1033600011884FF080480026D8F82430FB180093CD
:1033700007F1FF3AB346A36AABB91AF1030F06D9B6
:1033800039462046FFF796FF68B1002305E0D8F8DC
:103390002410009A511A8F42F3D283F311883046D9
:1033A00003B0BDE8F08FA06AE36AA9EB06021B1A1E
:1033B000934228BF1346402B1CD905F1400355F812
:1033C000042B40F8042B9D42F9D1A36A4033A36239
:1033D0004036A26AE36A9A4204D3E169204604397E
:1033E000FFF782FF8BF311884E45D8D2202383F359
:1033F0001188C0E71A4629460193FDF703FC019B9B
:10340000A26A1A441D44A2621E44E2E702694369AB
:103410009A4203D1C3681BB9184670470023FBE7E3
:10342000836A002BF8D0043B9B1AF5D01360C36865
:10343000013BC360C3691A44836902619A4224BF95
:10344000436A0361002383620123E5E710B50A4460
:103450000024C361029B006040608460C1608161A0
:1034600041610261036210BD08B5826943699342FC
:1034700001D1826882B98268013282605A1C42613D
:103480001970426903699A4201D3C36843610021FC
:10349000FDF7EEFE002008BD4FF0FF3008BD000034
:1034A00070B5202304460E4683F31188A568A5B1A4
:1034B000A368A269013BA360531CA361157822692C
:1034C000934224BFE368A361E3690BB120469847A8
:1034D000002383F31188284670BD31462046FDF74E
:1034E000B7FE0028E2DA85F3118870BD2DE9F04FB0
:1034F0001E4685B004460F469046D0F81C90202307
:1035000083F311884FF080420025526A0293B2186B
:103510000192AA4606F1FF3BA3680BB3A368013BE7
:10352000A360A369591CA1611B783B702369A16941
:10353000994224BFE368A3617A1CB9F1000F03D05C
:1035400003922046C847039A8AF31188B8F101080C
:1035500005F1010518D0029B83F311881746DBE7BC
:103560001BF1030F07D931462046FDF771FE0028F5
:10357000D2D0002306E04FF08042516A019A511ADE
:103580008E42F1D283F31188284605B0BDE8F08F52
:10359000C16081614161C3611144009B0060406072
:1035A0008260016103627047F8B504460E46174613
:1035B000202383F31188A568A5B1A368013BA3600C
:1035C00063695A1C62611E70236962699A4224BF52
:1035D000E3686361E3690BB120469847002080F3FC
:1035E0001188F8BD39462046FDF732FE0028E2DAA0
:1035F00085F31188F8BD0000836942699A4210B5CD
:1036000001D182687AB98268013282605A1C826173
:103610001C7803699A4201D3C36883610021FDF7D6
:1036200027FE204610BD4FF0FF3010BD2DE9F04FB2
:103630001E4685B004460F469046D0F81C902023C5
:1036400083F311884FF080420025526A0293B2182A
:103650000192AA4606F1FF3BA3680BB3A368013BA6
:10366000A36063695A1C62613978197023696169C2
:10367000994224BFE36863617A1CB9F1000F03D05B
:1036800003922046C847039A8AF31188B8F10108CB
:1036900005F1010518D0029B83F311881746DBE77B
:1036A0001BF1030F07D931462046FDF7D1FD002855
:1036B000D2D0002306E04FF08042516A019A511A9D
:1036C0008E42F1D283F31188284605B0BDE8F08F11
:1036D00000F1604300F01F02400903F56143090156
:1036E0008000C9B200F1604083F8001300F561402A
:1036F00001239340C0F8803103607047124B0021D2
:103700001A694FF0FF321A61196158695A6159619B
:10371000186A60F0805018621962586A5A620B4A3F
:103720005962106840F480701060186F00F44070A7
:10373000B0F5007F1EBF4FF48030186719675368DB
:1037400023F400735360704700380240007000405B
:10375000354B364A1A64364A4FF4404111601A68B4
:1037600042F001021A601A689207FCD59A6822F0AA
:1037700003029A609A689A602B4B19469A6812F075
:103780000C02FBD1186800F0F90018609A601A6802
:1037900042F480321A600B689B03FCD54B6F43F0F8
:1037A00001034B67204B5A6F9007FCD5214A5A60A2
:1037B0001A6842F080721A601D4B1A465968490413
:1037C000FCD5196841F4803119605368D803FCD5E1
:1037D000136843F400331360154A53689903FCD50A
:1037E000114B1A689201FCD5134A9A6040F20112FB
:1037F000C3F88C200022C3F89020104A40F209310F
:1038000011609A6842F002029A60074B9A6802F0CF
:103810000C02082AFAD15A6C42F480425A645A6E59
:1038200042F480425A66704700380240000400109B
:1038300000700040186C400900948838003C024039
:103840004B6843608B688360CB68C3600B694361DE
:103850004B6903628B6943620B6803607047000029
:10386000214B0246186B10B540F2FF7420431863D9
:10387000196D1E48214319651146FFF7E1FF1C48E9
:1038800002F11C01FFF7DCFF1A4802F13801FFF7D3
:10389000D7FF194802F15401FFF7D2FF174802F190
:1038A0007001FFF7CDFF164802F18C01FFF7C8FF4A
:1038B000144802F1A801FFF7C3FF134802F1C40145
:1038C000FFF7BEFF114802F1E001FFF7B9FF104812
:1038D00002F1FC01FFF7B4FF0E4802F58C71BDE860
:1038E0001040FFF7ADBF00BF0038024000000240AB
:1038F0000004024000080240000C02400010024098
:103900000014024000180240001C02400020024047
:10391000002402400028024080EA0102844612F09E
:10392000030F4FD111F0030F32D14DF8044D11F0B8
:10393000040F51F8043B0BD0A3F101329A4312F06B
:10394000803F04BF4CF8043B51F8043B16D100BF44
:1039500051F8044BA3F101329A4312F0803FA4F1D5
:1039600001320BD14CF8043BA24312F0803F04BF5C
:1039700051F8043B4CF8044BEAD023460CF8013BC9
:1039800013F0FF0F4FEA3323F8D15DF8044B704773
:1039900011F0010F06D011F8012B0CF8012B002AB1
:1039A00008BF704711F0020FBFD031F8022B12F0A0
:1039B000FF0F16BF2CF8022B8CF8002012F47F4F5B
:1039C000B3D1704711F8012B0CF8012B002AF9D163
:1039D000704700BF121012131211000000104100B6
:1039E00001105A00F8210220301102209411022007
:1039F00053544D3332463F3F3F3F3F3F0053544DBA
:103A0000333246375B347C355D780053544D333266
:103A100046375B367C375D7800000000C112000835
:103A2000AD120008E9120008D5120008E1120008E2
:103A3000CD120008B9120008A5120008B913000839
:103A4000A5130008E1130008CD130008D9130008DE
:103A5000C5130008B11300089D1300080000000002
:103A6000010000000000000000000000FD17000839
:103A7000D91A0008751B00084000400018110220E8
:103A8000181102200100000028110220800000000F
:103A900040010000050000007573625F70756D7075
:103AA0000000000000960000000000000000000080
:103AB0000000000000000000000000000000802A5C
:103AC00000000000AAAAAAAA00000000FFFF000050
:103AD0000000000000A00A0000000000000000003C
:103AE000AAAAAAAA00000000FFFF00000000000030
:103AF000000000000000000000000000AAAAAAAA1E
:103B000000000000FFFF00000000000000000000B7
:103B10008029000000000000AAAAAAAA80140000C0
:103B2000FFFF00000070700700000000008002002E
:103B300000000000AAAAAAAA00400100FFFF00009E
:103B400000000080080000000000000000000000ED
:103B5000AAAAAAAA00000000FFFF000000000000BF
:103B6000000000000000000000000000AAAAAAAAAD
:103B700000000000FFFF0000000000000000000047
:103B80000000000000000000AAAAAAAA000000008D
:103B9000FFFF000000000000000000000000000027
:103BA00000000000AAAAAAAA00000000FFFF00006F
:103BB0000000000000000000000000000000000005
:103BC00000000000000000000000000000000000F5
:103BD00000000000000000000000000000000000E5
:103BE00000000000000000000000000000000000D5
:103BF0000200000000000000D51500083D16000876
:103C00004000400088260220982602200200000082
:103C10000000000003000000000000007D16000806
:103C20000000000010000000A82602200000000094
:103C30000100000000000000280E02200101020027
:103C400025424F41524425002553455249414C25B8
:103C500000637562652D6F72616E67650030313289
:103C60003334353637383941424344454600000045
:103C700048657820546563686E6F6C6F6779204C77
:103C8000696D697465640050726F6669434E4320C4
:103C900043554245204F72616E676520424C0000DB
:103CA000E92A00085129000841150008CD2A00081A
:103CB00043000000B83C000809024300020100C0B4
:103CC0003209040000010202010005240010010570
:103CD00024010001042402020524060001070582D4
:103CE000030800FF09040100020A000000070501A3
:103CF00002400000070581024000000012000000A1
:103D0000043D00081201100102000040AE2D011018
:103D10000002010203010000040309040080000006
:103D20000080000000800000008000000000020011
:103D30000000040000000400000004000000040073
:103D40000000040000000400000004006D61696EC2
:103D5000000000006C3D000850290220482B022082
:103D600001000000352E00080000000069646C6549
:103D70000000000000000000FF0000000000000044
:103D8000F03900083F00000049040000FD39000838
:103D90003F000000510400000B3A00083F00000003
:103DA000009600000000080004000000183D000814
:103DB0000000000000000000000000000000000003
:083DC0000000000000000000FB
:00000001FF
